:100000007BC09FC09EC09DC09CC0A0C09AC099C02C
:1000100098C097C096C095C094C093C092C07445D4
:1000200079467D47824887498B60906194629963E5
:100030009D64A265A766AB67B068B469B980BE81EC
:10004000C282C783CB84D084D484FF210000000007
:1000500000000000000000000000000000000000A0
:100060000000000000000000000000000000000090
:100070002167B1FF030405070A0E1319212B36432C
:1000800053657990AAC6E6FFFFFFFFFFFFFFFFFF62
:10009000FFFFFFFFFFFFFFFFFFFFFF00000000006B
:1000A0000000000000000000000000000000000050
:1000B00008121C2834414E5C6B7C8FA3B8CFE6FF3E
:1000C000FFFFFF0028000628000617280006111C65
:1000D0002800060E171F2800060C131A21280014EA
:1000E00028EA00EAF406142800EA060C131D28008A
:1000F00006132000F4EA280011241FBECFE5D2E049
:10010000DEBFCDBF20E0A0E6B0E001C01D92A53764
:10011000B207E1F7E6E7F0E085E5808781E08383D9
:10012000148212828683118288E081878FE482871D
:10013000E0E6F0E08DEF87838EEF8583712C98D019
:100140008DC25ECF1BBC19BC18BC0895189525B78D
:10015000277E25BF29B7226029BF21E022BF019752
:1001600028F020E188952150E9F7F9CF089588EE2D
:1001700093E0EDCF369A3699FECF85B10895CF93AF
:10018000C72D81E0870D8F73782E662D90E058D2B1
:100190006FEF8C2F90E0CF9153C2FF920F931F937C
:1001A000CF93DF93F82E07E710E0CEE7D0E0F11011
:1001B00005C0CE013DD2F801808304C0F801608102
:1001C000CE013ED221970F5F1F4FC437D10579F77B
:1001D000DF91CF911F910F91FF900895D0DF81E0C3
:1001E000DCCF811101C0AECF815090E0FC01E45B17
:1001F000FF4FE491EBBDFC01EC58FF4FE491E9BDEA
:10020000FC01E456FF4F849188BD08950F931F931E
:10021000CF93C82F8B01CC2359F08AE0E2DFC801CD
:1002200096DF90DFC80193DFC80191DFC150F3CFA3
:10023000CF911F910F9108951F93CF93DF938FEA72
:1002400087B986EC86B910E1C0E0D0E085E090E0A7
:100250007EDF90DFC80FD11D1150C1F7CE0124E021
:10026000969587952A95E1F7DF91CF911F91089593
:100270001092750083EA87B986EC86B93699FECF6D
:10028000369A3699FECF85B18095582E87E790E053
:10029000CFD1853519F0612CA1DF11C0712C872DCC
:1002A00090E0C6D1682E8F3F19F080E076DF07C05E
:1002B000872D91E0970D792E803488F3F6CF209129
:1002C0007F00C091790010917A0080917700882397
:1002D00019F010E0C0E029E02F5F90E040E050E02E
:1002E000A4ECB0E0222379F0BD016F5F7F4FFB01EA
:1002F0003197E491EE2319F0962F9A1BF6CF2150F7
:10030000AD01DB01EFCF092F6C2F70E0A92FB0E01A
:10031000E02FF0E0112321F09D012E1B3F0B05C0C3
:100320009F0121503109260F371F3197E40FF51F28
:10033000F49027593F4FF901F082015049F79C0F83
:1003400090938100CC2371F0112329F0292F30E004
:100350002150310902C020E030E0F901E759FF4F98
:1003600041E0408323E0290F322F3150E32FE91B76
:10037000F0E0EC50FF4FE491A32FB0E0A759BF4F3E
:10038000EC933913F2CFE22FF0E0E859FF4F31E060
:10039000509169004081541330E0231B2093820068
:1003A000362D353FE8F5452D4134B0F4809183007A
:1003B0008F3F29F4809175008093830006C081E00F
:1003C000860D682E891708F0612C809183008F5F5D
:1003D0008F718093830024C0309175003093830027
:1003E0004F3AC0F430917C00332311F0882339F068
:1003F00081E0860D682E891798F0612C11C0862D3A
:100400006916D9F3662019F08150682E09C0215071
:10041000622E06C08111F1CF80917800882369F3A4
:100420008FEF8DBD80E68CBD8FE384BB8BE187BBF6
:1004300088EE88BB81E083BF91EA9ABD80BF85B713
:10044000806285BF789497B986EC86B9C62DC53F82
:1004500010F0612C3CC080918300803138F4E62D8F
:10046000F0E0E759FF4FC081DC2F31C080DE809182
:10047000750080938300C7E7D0E000E010E0FF2420
:10048000F39481E0800F0F5F1F4F98819F3F29F405
:10049000219608301105A9F7E2CF6DE570E0B6DED0
:1004A000F801E05AFF4F608088818F25888396DEAF
:1004B0006FE070E080E2AADE88818F258883612C5E
:1004C0008DDE55DE80917700882311F3C8CF57DE8B
:1004D00010E0F12C81EAE82E96ECD92ECC24CA94B7
:1004E000CA3E91F401E0802F7CDE88E290E02FDEAE
:1004F0000F5F0932C1F708E2802F73DE88E290E0D7
:1005000026DE0150C9F754C0C43F51F584E690E09F
:100510001EDE30DE90E0292F30E0F901E25EFF4F71
:10052000E491E81710F49E5FF6CFF901E15EFF4F0A
:1005300004916DE770E0802F82958695877066DE66
:100540008EEE92E004DE65E070E081E05FDE85E63D
:1005500094E0FDDD6DE770E0802F8F7157DE0DC0F8
:10056000CE3F71F400E000937F0038DE6AEF70E068
:1005700081E04CDE0F5F0930B1F7F9DDF8DD18C01E
:10058000CD3F39F58FEF8093800028DE8AE029DEA9
:10059000EEDDEDDD88E225DE4FDE809380001EDE9D
:1005A000E6DDE5DDF9CFD531F8F484EF91E0CFDD7C
:1005B0008091750080938300DDDD823808F036C0BD
:1005C0001F5F183008F48CCFD932A8F010E0D4E1C6
:1005D000C4E18D2F06DE30DEE7B8D6B8F3949091F3
:1005E0008000891710F3DFCFF4E1FF15F0F6C09219
:1005F0007500D4E1DACFD23030F08D2F8695869514
:10060000D695D80F12C09EDD85B7877E806185BFE5
:10061000F89485B7846885BF8B7F85BF85B7806276
:1006200085BF889585B78F7D85BFCD2F10E058CFCA
:10063000E199FECF9FBB8EBBE09A99278DB30895B9
:10064000262FE199FECF1CBA9FBB8EBB2DBB0FB6E8
:10065000F894E29AE19A0FBE01960895F894FFCFBC
:00000001FF
